:020000040000FA
:0200000058D0D6
:020008002BD0FB
:08001800D8CF01F0E8CF00F0A1
:10002000E0CF02F0EACF03F0E9CF04F09EAA02D0BD
:100030009DBA1FD09EA802D09DB801D0FF0040A25B
:1000400002D09D9802D0BBD8AD6E04C0E9FF03C0BA
:10005000EAFF02C0E0FF00C0E8FF01C0D8FF1000C7
:10006000EACF05F0E9CF06F0A1A202D0A0B2F3D00A
:10007000FF00ABB207D0ABB40BD040B410D0AE5041
:1000800081D8E3D7AB98AB881280FA0E5BD8DDD766
:10009000AE50AB98AB881280FB0E54D8D6D7AE507A
:1000A0001280FB0E4FD8D1D706C0E9FF05C0EAFF8A
:1000B0001100896A8A6A8B6A926A936AC00E946E8A
:1000C000070EC16EC26A926A106A116A126A8B8048
:1000D0000E68FF0EE82E6AEF00F00E2E69EF00F0BA
:1000E0008B90E00EDE6FDF6F00EE00F010EE00F0A0
:1000F00004D8ACD8B5EC01F0FDD7C00E94124F0E69
:10010000AF6E240EAC6E900EAB6E406A09D811D85B
:10011000300E9D6E000E9F6ED08EC00EF26E1200DD
:10012000000E446E466E4C0E456E476E4090408207
:100130001200000E486E4A6E5C0E496E4B6E409483
:10014000408612009D9840B01BD046C0EAFF47C0D1
:10015000E9FFEE6E000EEA6205D05C0EE96202D0A5
:1001600000EE4CF0EACF46F0E9CF47F0445046624B
:1001700004D04550476201D0408040929D881200D3
:100180009D88120040B41AD04AC0EAFF4BC0E9FF74
:10019000EE6E000EEA6205D06C0EE96202D000EE4F
:1001A0005CF0EACF4AF0E9CF4BF048504A6204D005
:1001B00049504B6201D0408440961200120040B278
:1001C0001CD044C0EAFF45C0E9FFEECF43F0000E6B
:1001D000EA6205D05C0EE96202D000EE4CF0EACF94
:1001E00044F0E9CF45F04650446204D047504562A0
:1001F00001D04082409043501200000C9D9A40B6BE
:100200001DD048C0EAFF49C0E9FFEECF42F0000E22
:10021000EA6205D06C0EE96202D000EE5CF0EACF33
:1002200048F0E9CF49F04A50486204D04B50496247
:1002300001D04086409442509D8A12009D8A000C55
:1002400040B61200DBDF7EDFFBD71200010EB16E7D
:10025000A282A0821200A192500EB26EB36810501A
:10026000896E11508A6E12508B6E00EE00F010EE07
:1002700000F0F86ADE51DF5D17E0DEC0E9FF080E2E
:10028000DE27DE5102E1E00EDE6FEE50100FE826B1
:10029000E16EE26AEE50E66EEE50E66EEE5010123F
:1002A000EE501112EE501212210604E2200602E274
:1002B00021681094230604E2220602E223681092C9
:1002C000250604E2240602E225681090270604E2CF
:1002D000260602E227681096290604E2280602E2B2
:1002E000296810982B0604E22A0602E22B68000017
:1002F0002D0604E22C0602E22D6800002F0604E21F
:100300002E0602E22F680000310604E2300602E207
:100310003168119A330604E2320602E2336811981A
:10032000350604E2340602E235681196370604E227
:10033000360602E237681194390604E2380602E212
:10034000396811923B0604E23A0602E23B6800007B
:100350003D0604E23C0602E23D6800003F0604E27E
:100360003E0602E23F6800009FD640B6120046DF1C
:10037000076E07AE0CD0086E000E0B6A08AC04D0F6
:1003800008AA010E0C6E02D0020E0C6E12000B6653
:1003900001D004D007C00AF00B6A08D007C009F0EA
:1003A0000B2A0B500C5C01E0120012009D0E085C41
:1003B00004E08D0E085C4FE012000A504CE00F0E76
:1003C000F76E09C0F6FF0800F55032E0F5040F6E35
:1003D00020EE00F0DFC0D9FFDE6E0A500A24F66E70
:1003E0000F50100FF76E0900F5CF0EF00900F55011
:1003F000DE6E0E50DE6E0E0EF76E0F500F240F24C1
:100400000F24F66E0900F550DE6E0900F550DE6E21
:100410000900F550DE6EDE6EDE6ED95003E0D9CFF6
:0A042000DFF01200E00EDF6F1200A3
:10043000640E095C23E0650E095C22E0660E095C2F
:1004400021E0670E095C20E0680E095C1FE0690E80
:10045000095C1EE01200640E095C1CE0650E095C7C
:100460001BE0660E095C1AE0670E095C18E0680E76
:10047000095C16E0690E095C15E01200108A120092
:10048000118E1200118C120011801200128A1200BB
:1004900012881200109A1200119E1200119C1190E5
:0804A000129A120012981200DA
:100E000004000000020000000100000008000000D3
:100E100010000000200000000080000000400000E2
:100E20000020000000100000000800000004000086
:100E3000000200000001000000002000000010007F
:100F000000000000000000000000000000000000E1
:100F100000000000000000000000000005040302C3
:100F200001000000000000000000000000000000C0
:100F300000000000000000000000000000000000B1
:100F40000000000000000000000000000D0C0B0A73
:100F50000900000000000000000000000000000088
:100F6000000000000607080E00000000000000005E
:100F70000000000000000000000000000000000071
:1010000000003200510070009000AF00CE00EE00F2
:101010000D012C014C016B018A01AA01C901E801F3
:1010200008022702460266028502A402C402E30205
:10103000030322034103610380039F03BF03DE0315
:10104000FD031D043C045B047B049A04B904D90429
:10105000F80417053705560576059505B405D4053A
:10106000F30512063206510670069006AF06CE064C
:10107000EE060D072C074C076B078A07AA07C9075E
:10108000E90708082708470866088508A508C4086E
:10109000E308030922094109610980099F09BF0981
:1010A000DE09FD091D0A3C0A5B0A7B0A9A0ABA0A94
:1010B000D90AF80A180B370B560B760B950BB40BA5
:1010C000D40BF30B120C320C510C700C900CAF0CB7
:1010D000CE0CEE0C0D0D2D0D4C0D6B0D8B0DAA0DC8
:1010E000C90DE90D080E270E470E660E850EA50EDA
:1010F000C40EE30E030F220F410F610F800FA00FEC
:1011000000003200510070009000AF00CE00EE00F1
:101110000D012C014C016B018A01AA01C901E801F2
:1011200008022702460266028502A402C402E30204
:10113000030322034103610380039F03BF03DE0314
:10114000FD031D043C045B047B049A04B904D90428
:10115000F80417053705560576059505B405D40539
:10116000F30512063206510670069006AF06CE064B
:10117000EE060D072C074C076B078A07AA07C9075D
:10118000E90708082708470866088508A508C4086D
:10119000E308030922094109610980099F09BF0980
:1011A000DE09FD091D0A3C0A5B0A7B0A9A0ABA0A93
:1011B000D90AF80A180B370B560B760B950BB40BA4
:1011C000D40BF30B120C320C510C700C900CAF0CB6
:1011D000CE0CEE0C0D0D2D0D4C0D6B0D8B0DAA0DC7
:1011E000C90DE90D080E270E470E660E850EA50ED9
:1011F000C40EE30E030F220F410F610F800FA00FEB
:1012000000003200510070009000AF00CE00EE00F0
:101210000D012C014C016B018A01AA01C901E801F1
:1012200008022702460266028502A402C402E30203
:10123000030322034103610380039F03BF03DE0313
:10124000FD031D043C045B047B049A04B904D90427
:10125000F80417053705560576059505B405D40538
:10126000F30512063206510670069006AF06CE064A
:10127000EE060D072C074C076B078A07AA07C9075C
:10128000E90708082708470866088508A508C4086C
:10129000E308030922094109610980099F09BF097F
:1012A000DE09FD091D0A3C0A5B0A7B0A9A0ABA0A92
:1012B000D90AF80A180B370B560B760B950BB40BA3
:1012C000D40BF30B120C320C510C700C900CAF0CB5
:1012D000CE0CEE0C0D0D2D0D4C0D6B0D8B0DAA0DC6
:1012E000C90DE90D080E270E470E660E850EA50ED8
:1012F000C40EE30E030F220F410F610F800FA00FEA
:1013000000003200510070009000AF00CE00EE00EF
:101310000D012C014C016B018A01AA01C901E801F0
:1013200008022702460266028502A402C402E30202
:10133000030322034103610380039F03BF03DE0312
:10134000FD031D043C045B047B049A04B904D90426
:10135000F80417053705560576059505B405D40537
:10136000F30512063206510670069006AF06CE0649
:10137000EE060D072C074C076B078A07AA07C9075B
:10138000E90708082708470866088508A508C4086B
:10139000E308030922094109610980099F09BF097E
:1013A000DE09FD091D0A3C0A5B0A7B0A9A0ABA0A91
:1013B000D90AF80A180B370B560B760B950BB40BA2
:1013C000D40BF30B120C320C510C700C900CAF0CB4
:1013D000CE0CEE0C0D0D2D0D4C0D6B0D8B0DAA0DC5
:1013E000C90DE90D080E270E470E660E850EA50ED7
:1013F000C40EE30E030F220F410F610F800FA00FE9
:1014000000003200510070009000AF00CE00EE00EE
:101410000D012C014C016B018A01AA01C901E801EF
:1014200008022702460266028502A402C402E30201
:10143000030322034103610380039F03BF03DE0311
:10144000FD031D043C045B047B049A04B904D90425
:10145000F80417053705560576059505B405D40536
:10146000F30512063206510670069006AF06CE0648
:10147000EE060D072C074C076B078A07AA07C9075A
:10148000E90708082708470866088508A508C4086A
:10149000E308030922094109610980099F09BF097D
:1014A000DE09FD091D0A3C0A5B0A7B0A9A0ABA0A90
:1014B000D90AF80A180B370B560B760B950BB40BA1
:1014C000D40BF30B120C320C510C700C900CAF0CB3
:1014D000CE0CEE0C0D0D2D0D4C0D6B0D8B0DAA0DC4
:1014E000C90DE90D080E270E470E660E850EA50ED6
:1014F000C40EE30E030F220F410F610F800FA00FE8
:1015000000003200510070009000AF00CE00EE00ED
:101510000D012C014C016B018A01AA01C901E801EE
:1015200008022702460266028502A402C402E30200
:10153000030322034103610380039F03BF03DE0310
:10154000FD031D043C045B047B049A04B904D90424
:10155000F80417053705560576059505B405D40535
:10156000F30512063206510670069006AF06CE0647
:10157000EE060D072C074C076B078A07AA07C90759
:10158000E90708082708470866088508A508C40869
:10159000E308030922094109610980099F09BF097C
:1015A000DE09FD091D0A3C0A5B0A7B0A9A0ABA0A8F
:1015B000D90AF80A180B370B560B760B950BB40BA0
:1015C000D40BF30B120C320C510C700C900CAF0CB2
:1015D000CE0CEE0C0D0D2D0D4C0D6B0D8B0DAA0DC3
:1015E000C90DE90D080E270E470E660E850EA50ED5
:1015F000C40EE30E030F220F410F610F800FA00FE7
:1016000000003200510070009000AF00CE00EE00EC
:101610000D012C014C016B018A01AA01C901E801ED
:1016200008022702460266028502A402C402E302FF
:10163000030322034103610380039F03BF03DE030F
:10164000FD031D043C045B047B049A04B904D90423
:10165000F80417053705560576059505B405D40534
:10166000F30512063206510670069006AF06CE0646
:10167000EE060D072C074C076B078A07AA07C90758
:10168000E90708082708470866088508A508C40868
:10169000E308030922094109610980099F09BF097B
:1016A000DE09FD091D0A3C0A5B0A7B0A9A0ABA0A8E
:1016B000D90AF80A180B370B560B760B950BB40B9F
:1016C000D40BF30B120C320C510C700C900CAF0CB1
:1016D000CE0CEE0C0D0D2D0D4C0D6B0D8B0DAA0DC2
:1016E000C90DE90D080E270E470E660E850EA50ED4
:1016F000C40EE30E030F220F410F610F800FA00FE6
:1017000000003200510070009000AF00CE00EE00EB
:101710000D012C014C016B018A01AA01C901E801EC
:1017200008022702460266028502A402C402E302FE
:10173000030322034103610380039F03BF03DE030E
:10174000FD031D043C045B047B049A04B904D90422
:10175000F80417053705560576059505B405D40533
:10176000F30512063206510670069006AF06CE0645
:10177000EE060D072C074C076B078A07AA07C90757
:10178000E90708082708470866088508A508C40867
:10179000E308030922094109610980099F09BF097A
:1017A000DE09FD091D0A3C0A5B0A7B0A9A0ABA0A8D
:1017B000D90AF80A180B370B560B760B950BB40B9E
:1017C000D40BF30B120C320C510C700C900CAF0CB0
:1017D000CE0CEE0C0D0D2D0D4C0D6B0D8B0DAA0DC1
:1017E000C90DE90D080E270E470E660E850EA50ED3
:1017F000C40EE30E030F220F410F610F800FA00FE5
:1018000000003200510070009000AF00CE00EE00EA
:101810000D012C014C016B018A01AA01C901E801EB
:1018200008022702460266028502A402C402E302FD
:10183000030322034103610380039F03BF03DE030D
:10184000FD031D043C045B047B049A04B904D90421
:10185000F80417053705560576059505B405D40532
:10186000F30512063206510670069006AF06CE0644
:10187000EE060D072C074C076B078A07AA07C90756
:10188000E90708082708470866088508A508C40866
:10189000E308030922094109610980099F09BF0979
:1018A000DE09FD091D0A3C0A5B0A7B0A9A0ABA0A8C
:1018B000D90AF80A180B370B560B760B950BB40B9D
:1018C000D40BF30B120C320C510C700C900CAF0CAF
:1018D000CE0CEE0C0D0D2D0D4C0D6B0D8B0DAA0DC0
:1018E000C90DE90D080E270E470E660E850EA50ED2
:1018F000C40EE30E030F220F410F610F800FA00FE4
:1019000000003200510070009000AF00CE00EE00E9
:101910000D012C014C016B018A01AA01C901E801EA
:1019200008022702460266028502A402C402E302FC
:10193000030322034103610380039F03BF03DE030C
:10194000FD031D043C045B047B049A04B904D90420
:10195000F80417053705560576059505B405D40531
:10196000F30512063206510670069006AF06CE0643
:10197000EE060D072C074C076B078A07AA07C90755
:10198000E90708082708470866088508A508C40865
:10199000E308030922094109610980099F09BF0978
:1019A000DE09FD091D0A3C0A5B0A7B0A9A0ABA0A8B
:1019B000D90AF80A180B370B560B760B950BB40B9C
:1019C000D40BF30B120C320C510C700C900CAF0CAE
:1019D000CE0CEE0C0D0D2D0D4C0D6B0D8B0DAA0DBF
:1019E000C90DE90D080E270E470E660E850EA50ED1
:1019F000C40EE30E030F220F410F610F800FA00FE3
:101A000000003200510070009000AF00CE00EE00E8
:101A10000D012C014C016B018A01AA01C901E801E9
:101A200008022702460266028502A402C402E302FB
:101A3000030322034103610380039F03BF03DE030B
:101A4000FD031D043C045B047B049A04B904D9041F
:101A5000F80417053705560576059505B405D40530
:101A6000F30512063206510670069006AF06CE0642
:101A7000EE060D072C074C076B078A07AA07C90754
:101A8000E90708082708470866088508A508C40864
:101A9000E308030922094109610980099F09BF0977
:101AA000DE09FD091D0A3C0A5B0A7B0A9A0ABA0A8A
:101AB000D90AF80A180B370B560B760B950BB40B9B
:101AC000D40BF30B120C320C510C700C900CAF0CAD
:101AD000CE0CEE0C0D0D2D0D4C0D6B0D8B0DAA0DBE
:101AE000C90DE90D080E270E470E660E850EA50ED0
:101AF000C40EE30E030F220F410F610F800FA00FE2
:101B000000003200510070009000AF00CE00EE00E7
:101B10000D012C014C016B018A01AA01C901E801E8
:101B200008022702460266028502A402C402E302FA
:101B3000030322034103610380039F03BF03DE030A
:101B4000FD031D043C045B047B049A04B904D9041E
:101B5000F80417053705560576059505B405D4052F
:101B6000F30512063206510670069006AF06CE0641
:101B7000EE060D072C074C076B078A07AA07C90753
:101B8000E90708082708470866088508A508C40863
:101B9000E308030922094109610980099F09BF0976
:101BA000DE09FD091D0A3C0A5B0A7B0A9A0ABA0A89
:101BB000D90AF80A180B370B560B760B950BB40B9A
:101BC000D40BF30B120C320C510C700C900CAF0CAC
:101BD000CE0CEE0C0D0D2D0D4C0D6B0D8B0DAA0DBD
:101BE000C90DE90D080E270E470E660E850EA50ECF
:101BF000C40EE30E030F220F410F610F800FA00FE1
:101C000000003200510070009000AF00CE00EE00E6
:101C10000D012C014C016B018A01AA01C901E801E7
:101C200008022702460266028502A402C402E302F9
:101C3000030322034103610380039F03BF03DE0309
:101C4000FD031D043C045B047B049A04B904D9041D
:101C5000F80417053705560576059505B405D4052E
:101C6000F30512063206510670069006AF06CE0640
:101C7000EE060D072C074C076B078A07AA07C90752
:101C8000E90708082708470866088508A508C40862
:101C9000E308030922094109610980099F09BF0975
:101CA000DE09FD091D0A3C0A5B0A7B0A9A0ABA0A88
:101CB000D90AF80A180B370B560B760B950BB40B99
:101CC000D40BF30B120C320C510C700C900CAF0CAB
:101CD000CE0CEE0C0D0D2D0D4C0D6B0D8B0DAA0DBC
:101CE000C90DE90D080E270E470E660E850EA50ECE
:101CF000C40EE30E030F220F410F610F800FA00FE0
:101D000000003200510070009000AF00CE00EE00E5
:101D10000D012C014C016B018A01AA01C901E801E6
:101D200008022702460266028502A402C402E302F8
:101D3000030322034103610380039F03BF03DE0308
:101D4000FD031D043C045B047B049A04B904D9041C
:101D5000F80417053705560576059505B405D4052D
:101D6000F30512063206510670069006AF06CE063F
:101D7000EE060D072C074C076B078A07AA07C90751
:101D8000E90708082708470866088508A508C40861
:101D9000E308030922094109610980099F09BF0974
:101DA000DE09FD091D0A3C0A5B0A7B0A9A0ABA0A87
:101DB000D90AF80A180B370B560B760B950BB40B98
:101DC000D40BF30B120C320C510C700C900CAF0CAA
:101DD000CE0CEE0C0D0D2D0D4C0D6B0D8B0DAA0DBB
:101DE000C90DE90D080E270E470E660E850EA50ECD
:101DF000C40EE30E030F220F410F610F800FA00FDF
:101E000000003200510070009000AF00CE00EE00E4
:101E10000D012C014C016B018A01AA01C901E801E5
:101E200008022702460266028502A402C402E302F7
:101E3000030322034103610380039F03BF03DE0307
:101E4000FD031D043C045B047B049A04B904D9041B
:101E5000F80417053705560576059505B405D4052C
:101E6000F30512063206510670069006AF06CE063E
:101E7000EE060D072C074C076B078A07AA07C90750
:101E8000E90708082708470866088508A508C40860
:101E9000E308030922094109610980099F09BF0973
:101EA000DE09FD091D0A3C0A5B0A7B0A9A0ABA0A86
:101EB000D90AF80A180B370B560B760B950BB40B97
:101EC000D40BF30B120C320C510C700C900CAF0CA9
:101ED000CE0CEE0C0D0D2D0D4C0D6B0D8B0DAA0DBA
:101EE000C90DE90D080E270E470E660E850EA50ECC
:101EF000C40EE30E030F220F410F610F800FA00FDE
:101F000000003200510070009000AF00CE00EE00E3
:101F10000D012C014C016B018A01AA01C901E801E4
:101F200008022702460266028502A402C402E302F6
:101F3000030322034103610380039F03BF03DE0306
:101F4000FD031D043C045B047B049A04B904D9041A
:101F5000F80417053705560576059505B405D4052B
:101F6000F30512063206510670069006AF06CE063D
:101F7000EE060D072C074C076B078A07AA07C9074F
:101F8000E90708082708470866088508A508C4085F
:101F9000E308030922094109610980099F09BF0972
:101FA000DE09FD091D0A3C0A5B0A7B0A9A0ABA0A85
:101FB000D90AF80A180B370B560B760B950BB40B96
:101FC000D40BF30B120C320C510C700C900CAF0CA8
:101FD000CE0CEE0C0D0D2D0D4C0D6B0D8B0DAA0DB9
:101FE000C90DE90D080E270E470E660E850EA50ECB
:101FF000C40EE30E030F220F410F610F800FA00FDD
:020000040030CA
:0E000000FFFEFDFEFFFEFAFFFFFFFFFFFFFF0A
:00000001FF
